:030000000246199C
:0C46190078FFE4F6D8FD75816102466070
:101D7C0020000A3C2E2E2E3E004950436F6E6E659D
:101D8C0063745245510A004950436F6E6E6563741B
:101D9C00000A49504E6F41434B210A003E432C56DA
:101DAC002C52432CC0E4E0EFF2E5F020D1E8EDEA50
:101DBC00EEEC49500A003E432C4D41432C25303269
:101DCC0062583A25303262583A25303262583A25F8
:101DDC00303262583A25303262583A2530326258E5
:101DEC002C4D414320E0E4F0E5F10A003E432C5633
:101DFC0045522C20332E3220EEF2202573202573F1
:101E0C002CC2E5F0F1E8FF20495020ECEEE4F3EBB6
:101E1C00FF0A0041707220313820323030380031E6
:101E2C00303A35373A3232003E432C4C442C505227
:101E3C004F473A2020202020202020202020202026
:101E4C002020202020202020202020202020202086
:101E5C002020202020202020202020202020202076
:101E6C002020202020202020202020202020202066
:101E7C0020202020202020202CC4E0F2E020EFF0B5
:101E8C00EEF8E8E2EAE828F4E0E9EB290A003E2A59
:101E9C002C312CCEF1EDEEE2EDFBE520EFE0F0E0A5
:101EAC00ECE5F2F0FB20F1E5F2E5E2EEE3EE20E802
:101EBC00EDF2E5F0F4E5E9F1E00A003E412C4130A9
:101ECC00312C2562752E2562752E2562752E2562A4
:101EDC00752C495020E0E4F0E5F120E0E4E0EFF26D
:101EEC00E5F0E00A003E412C4130322C2562752E83
:101EFC002562752E2562752E2562752C495020E0C1
:101F0C00E4F0E5F120EEF1ED2E20F1E5F0E2E5F064
:101F1C00E00A003E412C4130332C2562752E25629F
:101F2C00752E2562752E2562752C495020E0E4F043
:101F3C00E5F120F0E5E72E20F1E5F0E2E5F0E00A2E
:101F4C00003E412C4130342C2562752E2562752EB5
:101F5C002562752E2562752CCCE0F1EAE020F1E5C6
:101F6C00F2E80A003E412C4130352C2562752E25B5
:101F7C0062752E2562752E2562752CD8EBFEE70A4C
:101F8C00003E2A2C312CC4EEEF2E20EFE0F0E0ECDA
:101F9C00E5F2F0FB20F1E5F2E5E2EEE3EE20E8ED10
:101FAC00F2E5F0F4E5E9F1E00A003E422C53303161
:101FBC002C2562752CC6E4E0F2FC20E7E0EFF0EE95
:101FCC00F1E020F1EEE5E4E8EDE5EDE8FF20EEF2DE
:101FDC0020F1E5F0E2E5F0E00A003E422C5330320D
:101FEC002C2562752CCEE1ECE5ED20F120F1E5F02D
:101FFC00E2E5F0EEEC20E1E5E720EAE2E8F2E0EDE4
:10200C00F6E8E90A003E422C5330332C2562752C3D
:10201C00CFE5F0E5E7E0EFF3F1EA20EFF0E820EFB1
:10202C00EEF2E5F0E520F1E2FFE7E820F120F1E542
:10203C00F0E2E5F0EEEC0A003E422C5330352C2554
:10204C0062752CCAE0EDE0EB20F8E8F0EEEAEEE287
:10205C00E5F8E0F2E5EBFCEDEEE3EE20EEE1ECE58D
:10206C00EDE00A003E532C5330362C2530326258AA
:10207C00253032625825303262582530326258256C
:10208C003032625825303262582C4D414320E0E406
:10209C00F0E5F120F8E8F0EEEAEEE2E5F8E0F2E542
:1020AC00EBFCEDEEE3EE20EEE1ECE5EDE00A003EBC
:1020BC00454E440A000A44756D705820202020209B
:1020CC00303020303120303220303320303420304A
:1020DC003520303620303720303820303920304110
:1020EC002030422030432030442030452030460000
:1020FC000A3A003A20000A000A44756D7044202008
:10210C00202020303020303120303220303320302D
:10211C0034203035203036203037203038203039DC
:10212C0020304120304220304320304420304520A4
:10213C00304600457272206B6579005264206565EB
:10214C0070726F6D0A005264204D454D0A00526446
:10215C0020436F64650A00577269746520436F648D
:10216C00650A0044656275674950204F4E0A004469
:10217C00656275674950204F46460A004465627592
:10218C006755736572204F6E0A004465627567551A
:10219C00736572204F46460A0044656275674D733D
:1021AC0067204F6E0A0044656275674D7367204F58
:1021BC0046460A00436F6E666967206C6F636B213D
:1021CC000A00577220656570726F6D0A00205361AA
:1021DC00766520656570726F6D210A0045727220FC
:1021EC004D414321004C6F61643E3E002A003C414E
:1021FC0030313D003C4130323D003C4130333D00FC
:10220C003C4130343D003C4130353D003C21003CEC
:10221C005330313D003C5330323D003C5330333D64
:0D222C00003C5330353D003C5330363D0042
:06515500015E00015C0098
:1050EB00C28E438910758BFF758DB7D2ABD28E22D2
:03001B000244FAA2
:1044FA00C0E0C083C082C0D0C28E758BFF758DB7F5
:10450A0020060675A61E75A6E1055CD202E55E6068
:10451A0002055EE55DD394014002155D0561E56122
:10452A00540F7048D20EE561543F7012D200906E5B
:10453A00C5E0600A04F0E0D394B44002D206906E5B
:10454A00C0E0600204F090693EE0600214F0906EF0
:10455A00C6E0D394014003E014F0300502055FE59C
:10456A0060D394644004D20680020560E55BD3946C
:10457A00014002155BD28ED0D0D082D083D0E032F7
:1017AF00C2AFC20B7D027C007F071250758F26E5FA
:1017BF0026646060097D017F60124FC8D20BE4FD83
:1017CF00FC7F0B1250758F26E52630E6097D04E469
:1017DF00FF124FECD20B7D017C007F071250758FEB
:1017EF0026E5267008FD7FFF124FC8D20B300B0382
:1017FF00126000C288C2A8C2AA7589001243C590A0
:10180F006B837403F0A374CCF0E4906B82F01241FD
:10181F0099123193C206124C61D20BC20DC20C90B9
:10182F006DB07408F0906AEE7424F0E4A3F0906B3E
:10183F0078E0906AF0F0906B79E0906AF1F0906B3D
:10184F007AE0906AF2F0906B7BE0906AF3F0906B25
:10185F007CE0906AF4F0906B7DE0906AF5F0755D36
:10186F0001E4906DB1F0C207C208C209C20A124F5B
:10187F00A1200B19AF267E007D03123D49E4FF1214
:10188F0043157E1D7F7CE4FBFDFC123A56906EC51E
:10189F00E060037401F0E490693EF0F55F906DAF86
:1018AF00F0F5601250EB75A70775A61E75A6E1D26D
:1018BF00AFE4F56090693EE0700312285B906EC64E
:1018CF00E0B401119080007410F0E4906EC6F0D275
:1018DF000BC20CC20D908008E0F52630E405D2074C
:1018EF007410F0E52630E508D2099080087420F0D6
:1018FF00E52630E608D2089080087440F0E55FC313
:10190F0094034019908002E4F0908001F0908000E1
:10191F00F0E55F94064006E4F55F124C619080A0FD
:10192F00E07003124A529080B8E07003124ACC90D4
:10193F0080D0E07003124B46908000E070133007A8
:10194F0010123B5D906B6BEFF0D3940040031208C5
:10195F00E2908002E07006908000E06005D2050200
:10196F0018C0C205E4F55F90693EE060030218C03D
:10197F00200B12906DB2E0600C7E1D7F7E123C61D9
:10198F00E4906DB2F03009121237D7906B6BEFF015
:10199F00D394004005E0FF12510A200803021B24D4
:1019AF001234E1906B6BEFF070030218C0906BAFC5
:1019BF00E054BF247F7003021A8D147003021A655E
:1019CF0024026003021AC6200B077E1D7F85123C7E
:1019DF0061200F03021B24906B87E0FF7006906B52
:1019EF008BE06061906EBCE0FEB50722A3E0FF9034
:1019FF006B88E0B50718906EBEE0FF906B89E0B57D
:101A0F00070C906EBFE0FF906B8AE06F6037906BB2
:101A1F008BE06E6003021B24906EBDE0FF906B8C19
:101A2F00E06F6003021B24906EBEE0FF906B8DE0B1
:101A3F006F6003021B24906EBFE0FF906B8EE06F10
:101A4F006003021B24C203906DB17401F0120021D8
:101A5F00755D01021B24906EC5E060037401F09068
:101A6F006EB4E0FF906BB1E06F6003021B24906EC9
:101A7F00B4E004F0E4F55D906DAFF0021B24300389
:101A8F0003021B24906B7EE070030218C0906B8FD3
:101A9F00740AF012516AD203E4F55D906DAFF090C5
:101AAF006EC004F0E4906EB3F0A3F0200B677E1DC0
:101ABF007F93123C61805E906EC5E060037401F00D
:101ACF00300352906BAFE020E74B906BB1E0FF908B
:101ADF006EB3E0FE6F600D906EBBE07007EE146F9B
:101AEF0070338013906EB3E004F0906B6BE0FFD314
:101AFF0094044003124D8A90683A7482F0A37401E3
:101B0F00F0906BB1E090683CF07E687F3A7D0312F5
:101B1F0047B80218C0200303021C3CE55D70681231
:101B2F004E6FEF60237E6C7FAF906CB0E02404FDAE
:101B3F001247B8906EBBE07009906B8FE0F55D02B5
:101B4F0018C0E4F55D0218C0906EC0E0D3943C401D
:101B5F0036906EBBE07030906EC004F012514BE4C3
:101B6F00906CAFF0A37412F0906EB4E0906CB1F083
:101B7F00A374FDF090693F63A201906CB363A2015F
:101B8F007F12123085809E1251408F26E526B401B8
:101B9F001590683A7483F0E4A3F07E687F3A7D0273
:101BAF001247B80218C0E526D39401401C90683A3A
:101BBF007483F0A37401F0E52624FEA3F07E687F02
:101BCF003A7D031247B80218C0E55D640160030255
:101BDF0018C0906DAFE004F0200B077E1D7F9D12A3
:101BEF003C61906B8FE0C394C85004E02432F090B6
:101BFF006DAFE0C39405400DC203E4906DB1F012D8
:101C0F0000210218C07C6E7DBC906B83E0FAA3E0CC
:101C1F00FB7F021249CE7E6C7FAF906CB0E0240444
:101C2F00FD1247B8906B8FE0F55D0218C0E55D645B
:101C3F000160030218C0906DB1E014604624FE608D
:101C4F0042147003021D2F240460030218C0E4F530
:101C5F005F200F13906DB17404F0906DAFE05401DD
:101C6F00F0755D010218C09080027410F0E4906D61
:101C7F00B1F0906DAF04F0755DFA906EBC74FFF02B
:101C8F000218C0906EBCE07003021D19906CAF7407
:101C9F0080F0906CB17401F0E4A3F0A304F0A3748E
:101CAF0030F0A3747BF0E4F52674B62526F582E4B4
:101CBF00346CF583747DF074B72526F582E4346CAB
:101CCF00F583E4F0E5262407906CB0F07C6E7DBCC4
:101CDF00906B83E0FAA3E0FB7F021249CE7E6C7F0C
:101CEF00AFE5262409FD1247B8906EBBE0601B12CA
:101CFF00516AD203E4F55D906DAFF0906EC004F0C1
:101D0F00E4906EB3F0A3F00218C0300F07E4906DAB
:101D1F00B1F08006906DB17404F0755DFA0218C0D1
:101D2F009080027410F0755D05906DAFE06401FF57
:101D3F00F0906DB17401F0EF7019906B8BE0601340
:101D4F00FCA3E0FDA3E0FEA3E0FF906EBC12271DF5
:101D5F000218C0906B87E0FCA3E0FDA3E0FEA3E0B8
:0C1D6F00FF906EBC12271D0218C080FE01
:011D7B002245
:1008E200906BB0E0B444047F0180027F00906BAF54
:1008F200E0B447047E0180027E00EE5F604A906BA6
:1009020078E0906BB1F0906B79E0906BB2F0906B05
:100912007AE0906BB3F0906B7BE0906BB4F0906BED
:100922007CE0906BB5F0906B7DE0906BB6F0906BD5
:10093200B07452F0906AE863A2019080A863A201A9
:100942007F06123085021133906B6BE0C39408501E
:100952000302113C906B78E0FF906BB1E06F600393
:1009620002113C906B79E0FF906BB2E06F60030282
:10097200113C906B7AE0FF906BB3E06F6003021161
:100982003C906B7BE0FF906BB4E06F600302113C24
:10099200906B7CE0FF906BB5E06F600302113C90BE
:1009A2006B7DE0FF906BB6E06F600302113C906BD1
:1009B200B0E0B44415906AE8E0B4FF0E63A201907F
:1009C20080A863A2017F06123085906EC5E06003A5
:1009D2007401F0906EC67464F0906BB07452F09033
:1009E2006BAFE0646D6003020B417BFF7A1D79A857
:1009F20012229B7BFF7A1D79C2906B78E0F52FA3C0
:100A0200E0F530A3E0F531A3E0F532A3E0F533A33E
:100A1200E0F53412229B752FFF75301E75311F755C
:100A220032FF75331E75342B7BFF7A1D79F8122243
:100A32009B7BFF7A1E793412229B7BFF7A1E799A66
:100A420012229B7BFF7A1E79C7906B7EE0F52FA363
:100A5200E0F530A3E0F531A3E0F53212229B7BFFF3
:100A62007A1E79F1906B87E0F52FA3E0F530A3E0D1
:100A7200F531A3E0F53212229B7BFF7A1F791F909A
:100A82006B8BE0F52FA3E0F530A3E0F531A3E0F5A1
:100A92003212229B7BFF7A1F794D906B74E0F52F07
:100AA200A3E0F530A3E0F531A3E0F53212229B7BFF
:100AB200FF7A1F7970906B70E0F52FA3E0F530A3F9
:100AC200E0F531A3E0F53212229B7BFF7A1F798D8C
:100AD20012229B7BFF7A1F79B6A20FE433F52F1205
:100AE200229B7BFF7A1F79E6906EBBE0F52F1222E4
:100AF2009B7BFF7A207911906EC5E0F52F12229B25
:100B02007BFF7A207944A201E433F52F12229B7BEA
:100B1200FF7A207970906EB5E0F52FA3E0F530A34F
:100B2200E0F531A3E0F532A3E0F533A3E0F53412AA
:100B3200229B12393D7BFF7A2079BB12229B2290A5
:100B42006BAFE0644C70737E207FC1FBFDFC123AF8
:100B520056906BB7E0F527A3E0F528E4F52AE527E0
:100B6200906BB9F0A3E528F07E207FFC7C6B7DB909
:100B72007B02123A56E4F529852882852783E0FF15
:100B820074B92529F582E4346BF583EFF00528E585
:100B920028700205270529E529B410DC7E207FFF95
:100BA2007C6B7DB97B10123A56052AE52AC3941054
:100BB20040AC7E217F02123C6122906BAFE0646CFC
:100BC2007060F52B7E217F04FBFDFC123A56E4F5A2
:100BD2002AE4906BB9F0A3E52BF07E207FFC7C6BBE
:100BE2007DB97B02123A56E4F529A82BE6FF74B9C7
:100BF2002529F582E4346BF583EFF0052B0529E511
:100C020029B410E67E207FFF7C6B7DB97B10123AFF
:100C120056052AE52AC3940840B77E217F02123C7A
:100C22006122906BAFE0644B7061F52974A12529B4
:100C3200F582E4346BF583E0603274A12529F582F4
:100C4200E4346BF583E0F4602374A12529F582E492
:100C5200346BF583E0FF74B72529F582E4346BF534
:100C620083E0B507100529E529B408C090693E74F0
:100C720032F0021133906BAF7421F0300B0302118A
:100C8200337E217F3F123C61021133906BAFE0B49F
:100C9200521A200B077E217F47123C61906BAF7482
:100CA20072F07E6B7FAF7D0812473122906BAFE00E
:100CB20064497045200B077E217F52123C61906B84
:100CC200B7E0F527A3E0F528E4F5298528828527F2
:100CD20083E0FF74B92529F582E4346BF583EFF0E4
:100CE2000528E528700205270529E529B480DC7E60
:100CF2006B7FAF7D8A12473122906BAFE064437005
:100D020046200B077E217F5A123C61906BB7E0F5BB
:100D120027A3E0F528E4F529852882852783E49333
:100D2200FF74B92529F582E4346BF583EFF00528C9
:100D3200E528700205270529E529B480DB7E6B7F53
:100D4200AF7D8A12473122906BAFE0645A70532014
:100D52000B077E217F63123C61906BB7E0F527A3FE
:100D6200E0F5287C6B7DB97B80AF28AE27124E3B25
:100D7200E4F529852882852783E493FF74B9252920
:100D8200F582E4346BF583EFF00528E5287002055F
:100D9200270529E529B480DB7E6B7FAF7D8A124768
:100DA2003122906BAFE064446003020E35906BB762
:100DB200E0FF64447003021133EFB4310CC20B7EC6
:100DC200217F6F123C61021133906BB7E0B4300C9B
:100DD200D20B7E217F7B123C61021133906BB7E014
:100DE200B4320CD20C7E217F88123C610211339006
:100DF2006BB7E0B4330CC20C7E217F96123C6102C9
:100E02001133906BB7E0B4340CD20D7E217FA51262
:100E12003C61021133906BB7E0B4350CC20D7E21F8
:100E22007FB2123C61021133906BB7E0FF12001ED9
:100E320002113390693EE07013200B077E217FC0C0
:100E4200123C61906BAF7421F002113390693E74D1
:100E520032F0906BAFE0FFB45104C2AF80FEEF649A
:100E6200577045200B077E217FCE123C61906BB8F4
:100E7200E0906B6BF0E4F529906B6BE0FFE529C322
:100E82009F400302113374B92529F582E4346BF5CE
:100E920083E0FF906BB7E0252924E7F582E434690B
:100EA200F583EFF0052980D0906BAFE064536003C7
:100EB200020F57200B077E217FD9123C61906B787D
:100EC200E0FF9069F0E06F703C906B79E0FF906911
:100ED200F1E06F7030906B7AE0FF9069F2E0B50755
:100EE20024906B7BE0FF9069F3E0B50718906B7C70
:100EF200E0FF9069F4E0B5070C906B7DE0FF90692C
:100F0200F5E06F6016906BAF7421F0300B030211A5
:100F1200337E217FE8123C61021133E4F529E4F5C6
:100F22006074E72529F582E43469F583E0FDAF2991
:100F3200124EFC0529E529C394FE40E2C2AFE490BB
:100F42007FF0F0A3F0907FFD74AAF0A374FFF0A3EA
:100F52007455F080FE906BAFE0644F704C906BB7AD
:100F6200E0F527A3E0F528E5284527700A200B07BE
:100F72007E217FF1123C61200B077E217FF8123C1B
:100F820061E4F52974B92529F582E4346BF583E02F
:100F9200852882852783F00528E528700205270524
:100FA20029E529B480DE021133906BAFE0FFB4452E
:100FB20021906BB7E0FDA3E0907FF0CDF0A3EDF0C0
:100FC200C2AF907FFD74AAF0A374FFF0A37455F032
:100FD20080FEEF6465600302113C906BB7E0FFA3F3
:100FE200E0907FF0CFF0A3EFF0E4F527F528D3905F
:100FF2007FF1E09528907FF0E095274021E4F560AD
:101002002528FFE5273478FE7B80AD28AC27124ED9
:101012003B74802528F528E43527F52780D07E21EA
:101022007FFA12483FEF4E6020120003906B7EEF72
:10103200F0120003906B7FEFF0120003906B80EFD1
:10104200F0120003906B81EFF07E227F0012483F86
:10105200EF4E6020120003906B87EFF012000390B6
:101062006B88EFF0120003906B89EFF0120003908F
:101072006B8AEFF07E227F0612483FEF4E6020120D
:101082000003906B8BEFF0120003906B8CEFF01269
:101092000003906B8DEFF0120003906B8EEFF07EE9
:1010A200227F0C12483FEF4E6020120003906B74B7
:1010B200EFF0120003906B75EFF0120003906B7665
:1010C200EFF0120003906B77EFF07E227F1212484E
:1010D2003FEF4E6020120003906B70EFF01200039E
:1010E200906B71EFF0120003906B72EFF01200033D
:1010F200906B73EFF0E4F529E4F560E52904FF74E1
:10110200702529F582E4346BF583E0FD124EFC056F
:1011120029E529C3944340E0C2AFE4907FF0F0A3F5
:10112200F0907FFD74AAF0A374FFF0A37455F080D1
:0A113200FE7E6B7FAF7D081247318F
:01113C002290
:104E0300AE07EEC39430400BEED394395005EE2435
:104E1300D0FF22EEC39461400BEED394665005EEAF
:104E230024A9FF22EEC39441400BEED394465005D0
:084E3300EE24C9FF22AF0622A4
:10509200906AE7E004F07006906AE6E004F0906A35
:0A50A200E6E0FEA3E0FF124D4822F5
:10000300125092124E03EFC454F0FEC006125092E7
:08001300124E03D0E02FFF2282
:104BA900E4907005F0125092907006EFF0C39430C3
:104BB9004018E0FFD394395011907005E0243FF577
:104BC90082E43469F583EFF08011907005E0243FA9
:104BD900F582E43469F583E4F0800C907005E00413
:104BE900F0E0D3940840BE75320075330075340087
:0C4BF900E4F5357B017A69793F12333D09
:014C0500228C
:04483F008E2C8F2DFF
:10484300906AE6E4F0A374FFF0125092EF606EF406
:10485300606B852D82852C83E493B507EC752E015F
:10486300E52D252EF582E4352CF583E49360259020
:104873006AE7E0252EFF906AE6E03400FE124D4819
:10488300E52D252EF582E4352CF583E493B5070455
:10489300052E80CCE52D252EF582E4352CF583E419
:1048A3009370A6E52E24FFFFE434FFFE906AE7E051
:1048B3002FF0906AE6E03EF07E007F0122E4FEFFE7
:0148C30022D2
:104199007E227F1812483FEF4E70037F01227E2254
:1041A9007F1B12483FEF4E600C125092EF24D0242F
:1041B900FF920F8002D20F7E227F2112483FEF4EDD
:1041C900600C125092EF24D0906EBBF08005E49001
:1041D9006EBBF07E227F2712483FEF4E600C1250D3
:1041E90092EF24D0906EC5F08005E4906EC5F07E04
:1041F900227F2D12483FEF4E600C125092EF24D0CF
:1042090024FF92018002C201906B7863A201906E33
:10421900B563A2017F0612308530013B7E227F33D0
:1042290012483FEF4E6030120003906EB5EFF01266
:104239000003906EB6EFF0120003906EB7EFF01224
:104249000003906EB8EFF0120003906EB9EFF01210
:0A4259000003906EBAEFF07F002220
:104CBA00906DB0E0C3947C503D906DB0E0FE04F07E
:104CCA0074EE2EF582E4346AF583EFF0BF0A27907A
:104CDA006DB0E0FF04F074EE2FF582E4346AF583D8
:104CEA00E4F0906DB0E0FF1248C4906DB07408F023
:074CFA00906AEFE004F022D4
:104C61009080007480F0906B7063A201F583F582EF
:104C710063A2017F08123085906B7863A201908056
:104C81008863A2017F0A123085908092E4F0A374B8
:104C910032F0A37401F0906B82E0FF9080B1F0904C
:104CA10080E1EFF09080957455F0A3F0908000744E
:094CB10001F090800974F0F0227A
:104A5200908009E04410F09080A0E0706C9080A1FA
:104A62007482F09080A874FFF0A3F0A3F0A3F07F0B
:104A7200039080AEEFF07FCBA3EFF07F039080AC8A
:104A8200EFF0A374CBF09080007402F0906FF912F3
:104A9200272900000000906FF9E0908040F0906FAD
:104AA200FAE0908041F0906FFBE0908042F0906FCE
:104AB200FCE0908043F0A3E4F0A3F0A3F0A3F09015
:094AC2008018F0A3F0A3F0A3F0AA
:014ACB0022C8
:104B4600908009E04440F09080D17482F0906B83AD
:104B5600E0FF9080DEF0906B84E0FF9080DFF090C5
:104B660080027402F0906FFD122729000000009069
:104B76006FFDE0908058F0906FFEE0908059F090C5
:104B86006FFFE090805AF0907000E090805BF0A399
:104B9600E4F0A3F0A3F0A3F0908030F0A3F0A3F02C
:024BA600A3F07A
:014BA80022EA
:104ACC00908009E04420F09080B8E0706C9080B940
:104ADC007482F07F039080C6EFF07FCDA3EFF07F60
:104AEC00039080C4EFF0A374CDF09080C074FFF0FD
:104AFC00A3F0A3F0A3F09080017402F09070011267
:104B0C00272900000000907001E090804CF090701C
:104B1C0002E090804DF0907003E090804EF0907029
:104B2C0004E090804FF0A3E4F0A3F0A3F0A3F09086
:094B3C008024F0A3F0A3F0A3F023
:014B4500224D
:1049CE008C278D28A907EAFDE975F018A424ACFF01
:1049DE00E5F034808F82F583EDF0EBFDE975F0188C
:1049EE00A4FFAEF024ACFBEE34808B82F583A3EDF6
:1049FE00F08528828C83E0FDEF24A8FFEE3480FE44
:104A0E008F82F583EDF08528828C83A3E08F828ED2
:104A1E0083A3F0852882852783A3A3E0FDE975F0A3
:104A2E0018A424A8FFE5F03480FE8F82F583A3A39B
:104A3E00EDF08528828C83A3A3A3E08F828E83A3BF
:044A4E00A3A3F0220C
:064731008D2CAB07AA0667
:10473700908000E030E507906DB27401F022906F31
:10474700F9E0FCA3E0FDA3E0FEA3E0F5308E2F8D9A
:104757002E8C2DAE02AF038E838F8263A201E52FCD
:10476700540744C0F58385308263A201AF2C123011
:10477700F7E4FCFDFEE530252CF530EE352FF52F5F
:10478700ED352EF52EEC352DF52D908040E52DF0ED
:10479700A3E52EF0A3E52FF0A3E530F09080007499
:1047A70020F0AF30AE2FAD2EAC2D906FF912271D34
:0147B70022DF
:0647B8008D27AB07AA06E5
:1047BE00908002E030E507906DB27403F022906FA6
:1047CE00FDE0FCA3E0FDA3E0FEA3E0F52B8E2A8D19
:1047DE00298C28AE02AF038E838F8263A201E52A55
:1047EE00540744D0F583852B8263A201AF27123084
:1047FE00F7E4FCFDFEE52B2527F52BEE352AF52AF1
:10480E00ED3529F529EC3528F528908058E528F066
:10481E00A3E529F0A3E52AF0A3E52BF0908002741E
:10482E0020F0AF2BAE2AAD29AC28906FFD12271DBC
:01483E002257
:024315008F28EF
:10431700908001E030E509906DB27402F07F0022D1
:10432700907001E0FCA3E0FDA3E0FEA3E0F52C8E76
:104337002B8D2A8C29906EB563A201E52B54074477
:10434700C8F583852C8263A2017F0612310DE52C07
:104357002406F52CE4352BF52BE4352AF52AE4352C
:1043670029F529906DB363A201E52B540744C8F5DD
:1043770083852C8263A201AF2812310DE4FCFDFE78
:10438700E52C2528F52CEE352BF52BED352AF52ACE
:10439700EC3529F52990804CE529F0A3E52AF0A30F
:1043A700E52BF0A3E52CF09080017420F0AF2CAE44
:0D43B7002BAD2AAC2990700112271DAF28F4
:0143C40022D6
:103B5D009081E0E0F527052705270527052705278F
:103B6D0005270527052705270527908010E0F52A4D
:103B7D00A3E0F52BA3E0F52CA3E0F52D9081E1E07A
:103B8D00F5270527052705270527052705270527D8
:103B9D00052705270527908014E0F52EA3E0F52FC6
:103BAD00A3E0F530A3E0F531E530B52C08E531B5EE
:103BBD002D037F0022E4F527E530540744E0F5831B
:103BCD0085318263A201906BAF63A2017F08123130
:103BDD003D906BB163A201906AE863A2017F06126A
:103BED003085906BAFE0F528A3E0F529E4F527903B
:103BFD006BAFE0702AA3E024F8F527E530540744B5
:103C0D00E0F58385318274082582F582E43583F5EC
:103C1D008363A201906BAF63A201AF2712313DAE5A
:103C2D0028E4FCFDE5312529F531E5303EF530ED93
:103C3D00352FF52FEC352EF52E908014E52EF0A3B3
:103C4D00E52FF0A3E530F0A3E531F090800074404E
:033C5D00F0AF279E
:013C60002241
:1034E1009081E6E0F527052705270527052705270C
:1034F10005270527052705270527908028E0F52AB8
:10350100A3E0F52BA3E0F52CA3E0F52D9081E7E0F6
:10351100F52705270527052705270527052705275A
:1035210005270527052790802CE0F52EA3E0F52F30
:10353100A3E0F530A3E0F531E4F527E530B52C0A39
:10354100E531B52D05C20802364DE530540744F08A
:10355100F58385318263A201906BAF63A2017F087D
:1035610012313D906BAFE0F528A3E0F529E529453F
:103571002870099080027410F07F0022906EBCE0E8
:10358100FFF46030906BB1E06F6003023614906E0F
:10359100BDE0FF906BB2E06F7079906EBEE0FF907E
:1035A1006BB3E06F706D906EBFE0FF906BB4E06F36
:1035B1006031805F906BB1E0906EBCF0906BB2E0D7
:1035C100906EBDF0906BB3E0906EBEF0906BB4E086
:1035D100906EBFF0906BB5E0FFA3E0906B83CFF0EE
:1035E100A3EFF0906BAFE0702AA3E024F8F527E594
:1035F10030540744F0F58385318274082582F582C1
:10360100E43583F58363A201906BAF63A201AF2719
:1036110012313DAE28E4FCFDE5312529F531E530D7
:103621003EF530ED352FF52FEC352EF52EAF2DAEC5
:103631002CAD2BAC2AAB31AA30A92FA82ED312273F
:103641000C40099080027410F07F002290802CE5DC
:103651002EF0A3E52FF0A3E530F0A3E531F0908043
:06366100027440F0AF27E7
:013667002240
:1037D7009081E3E0F5270527052705270527052716
:1037E7000527052705270527052790801CE0F52ACB
:1037F700A3E0F52BA3E0F52CA3E0F52D9081E4E001
:10380700F527052705270527052705270527052761
:10381700052705270527908020E0F52EA3E0F52F43
:10382700A3E0F530A3E0F531E4F527E530B52C0A40
:10383700E531B52D05C209023922E530540744E8C0
:10384700F58385318263A20190683E63A2017F0EF2
:1038570012315390683EE0F528A3E0F529906846B9
:10386700E0FFF46045906EB5E0FEEF6E706EA3E08A
:10387700FF906847E06F7064906EB7E0FF9068480C
:10388700E06F7058906EB8E0FF906849E06F704C39
:10389700906EB9E0FF90684AE06F7040906EBAE0B2
:1038A700FF90684BE06F60048032D2D990683EE0A9
:1038B700702AA3E024F2F527E530540744E8F5839E
:1038C700853182740E2582F582E43583F58363A200
:1038D7000190683E63A201AF27123153AE28E4FC82
:1038E700FDE5312529F531E5303EF530ED352FF58C
:1038F7002FEC352EF52EAF2DAE2CAD2BAC2AAB31E0
:10390700AA30A92FA82ED312270C5006E52945283F
:1039170070099080017410F07F0022908020E52EBE
:10392700F0A3E52FF0A3E530F0A3E531F090800197
:053937007440F0AF2711
:01393C002268
:043C61008E2D8F2EE7
:103C6500908000E030E507906DB27401F022906F0E
:103C7500F9E0FCA3E0FDA3E0FEA3E0F5348E338D6F
:103C8500328C31E534FFE5335407FEE42FF530EE91
:103C950034C0F52F853082F5837423F00530E53087
:103CA5007002052F532FC7F582852F83740AF005FF
:103CB50030E5307002052F532FC7906B7863A20152
:103CC500852F8385308263A2017F061230F7740643
:103CD5002530F530E4352FF52F852D83852E82632C
:103CE500A201852F8385308263A2011230DBE4FCBB
:103CF500FDFE906FF9E0F8A3E0F9A3E0FAA3E02F49
:103D0500FFEE3AFEED39FDEC38FCEF2408FFE43E0A
:103D1500FEE43DFDE43CFC906FF912271D906FF920
:103D2500E0908040F0906FFAE0908041F0906FFB5A
:103D3500E0908042F0906FFCE0908043F09080002E
:033D45007420F0F7
:013D48002258
:0A3A56008E2C8F2D8C2E8D2F8B30BF
:103A6000908000E030E507906DB27401F022906F15
:103A7000F9E0FCA3E0FDA3E0FEA3E0F5368E358D72
:103A8000348C33E536FFE5355407FEE42FF532EE8E
:103A900034C0F531853282F5837423F00532E53286
:103AA000700205315331C7F582853183740AF00500
:103AB00032E532700205315331C7906B7863A20151
:103AC00085318385328263A2017F061230F7740646
:103AD0002532F532E43531F531852C83852D82632D
:103AE000A20185318385328263A2011230DB8F37D8
:103AF000EF2532F532E43531F531E5306017852EAA
:103B000083852F8263A20185318385328263A2017E
:103B1000AF301230F7E53724082530F530FFE4FCEC
:103B2000FDFEE5362FF536EE3535F535ED3534F558
:103B300034EC3533F533908040E533F0A3E534F0D1
:103B4000A3E535F0A3E536F09080007420F0AF36A1
:0C3B5000AE35AD34AC33906FF912271D78
:013B5C002246
:063FE8008E2D8F2E8D2F9F
:103FEE00908000E030E507906DB27401F022906F82
:103FFE00F9E0FCA3E0FDA3E0FEA3E0F5358E348DE1
:10400E00338C32E535FFE5345407FEE42FF531EEFF
:10401E0034C0F530853182F5837423F00531E531F6
:10402E00700205305330C7F582853083EBF00531D1
:10403E00E531700205305330C7906B7863A201856D
:10404E00308385318263A2017F061230F774062514
:10405E0031F531E43530F530852D83852E8263A21E
:10406E000185308385318263A201AF2F1230F77440
:10407E0008252FF52FFFE4FCFDFEE5352FF535EE77
:10408E003534F534ED3533F533EC3532F532908089
:10409E0040E532F0A3E533F0A3E534F0A3E535F0C7
:1040AE009080007420F0AF35AE34AD33AC32906FEB
:0440BE00F912271DAF
:0140C20022DB
:0248C4008F4023
:1048C600908000E030E507906DB27401F022906FA1
:1048D600F9E0FCA3E0FDA3E0FEA3E0F5448E438DE2
:1048E600428C41E544FFE5435407FEE42FFFEE34D6
:1048F600C0906AEE63A201F5838F8263A201AF4086
:104906001230F7E4FCFDFEE5442540F544EE354360
:10491600F543ED3542F542EC3541F541908040E5F1
:1049260041F0A3E542F0A3E543F0A3E544F090800F
:10493600007420F0AF44AE43AD42AC41906FF91223
:02494600271D2B
:01494800224C
:063D49008E2A8F2BAB0552
:103D4F00908000E030E507906DB27401F022906F23
:103D5F00F9E0FCA3E0FDA3E0FEA3E0F5318E308D8A
:103D6F002F8C2EE531FFE5305407FEE42FF52DEEB5
:103D7F0034C0F52C852D82F5837423F0052DE52DA8
:103D8F007002052C532CC7F582852C83EBF0052D83
:103D9F00E52D7002052C906B7863A201852C83852D
:103DAF002D8263A2017F061230F77406252DF52DA3
:103DBF00E4352CF52C532CC7E52A852D82852C83D1
:103DCF00F0052DE52D7002052C532CC7F582852C9F
:103DDF0083E52BF0052DE52D7002052C532CC7E53F
:103DEF0031240AF531E43530F530E4352FF52FE481
:103DFF00352EF52E908040E52EF0A3E52FF0A3E5AC
:103E0F0030F0A3E531F09080007420F0AF31AE3088
:0A3E1F00AD2FAC2E906FF912271D95
:013E29002276
:1043C500E4F527E5272401FFE433FE124D48747018
:1043D5002527F582E4346BF583EFF00527E527C340
:1043E500943F40DFE4F527E527247FFFE433FE1201
:1043F5004D4874672527F582E43469F583EFF07439
:10440500672527F582E43469F583E0FF6003B4FF8F
:104415001D74672527F582E43469F5837420F074EB
:10442500682527F582E43469F583E4F080090527DA
:10443500E527C3948040B0E49069E6F0F527AF27FF
:104445007E00124D4874E72527F582E43469F5832B
:0B445500EFF00527E527C394FE40E3CD
:014460002239
:10505500E4FDFCC3ED9FEC9E5015E4FBFA0BBB0091
:0F506500010ABA01F8BB90F50DBD00010C80E403
:015074002219
:0D5119004390014390025390FE5390FD22FD
:0D5126005390FD5390FE43900243900122F0
:0E50FB005390FD439002E5905408FF5390FD42
:015109002283
:0D5133005390FD4390014390025390FD22E4
:07515C00AE071FEE70FA22FE
:024ED000AD072C
:104ED200E4FC5390FDEDA804088002C333D8FC30F3
:104EE200E70543900180035390FE7F0512515C4316
:094EF20090020CBC08DC5390FD99
:014EFB002294
:104F5000E4FF5390FD7E07439002E59030E00D742E
:104F600001A806088002C333D8FC42075390FD1EF7
:084F7000C3EE6480948050DF61
:014F78002216
:104EFC00AB05AA071251197FA0124ED01250FBAF6E
:104F0C0002124ED01250FBAF03124ED01250FB12B5
:0A4F1C0051267F0A7E001250552234
:044D4800AB07AA0605
:104D4C00C3EB94FFEA9400400DE42BF58274773AA0
:104D5C00F583E493FF221251197FA0124ED012500A
:104D6C00FBAF03124ED01250FB1251197FA1124E01
:0D4D7C00D01250FB124F501251331251262D
:014D89002207
:024E3B008B2CBE
:104E3D00A2AF9220C2AF85A22D53A2FE8E838F8288
:104E4D0005A28C838D827409123181E52C53A2FE4B
:104E5D0043A22012318353A2DF852DA2A22092AF4F
:014E6D00FF45
:014E6E002221
:10507500A2AF9220C2AF8C838D82EF12318143A201
:0C5085002012318353A2DFA22092AFFF63
:0150910022FC
:024FC8008F2731
:104FCA00A2AF9220C2AFE4F5838D827406123181BA
:104FDA00E52743A22012318353A2DFA22092AF7F9A
:014FEA0001C5
:014FEB0022A3
:024FEC008F270D
:104FEE00A2AF9220C2AFE4F5838D82740A12318192
:104FFE00E52743A22012318353A2DFA22092AF7F76
:01500E0001A0
:01500F00227E
:102FAA00A907E7FFA805EF93C3966008403B74FCA6
:102FBA002FFF80F00F08EF93C3966008402B74FB35
:102FCA002FFF80E00F08EF93C3966008401B74FA46
:102FDA002FFF80D00F08EF93D3966008400B74F947
:102FEA002FFF80C01F1F1F1F1FEF54FEF80303F798
:102FFA00E893FC08E893FD08E893FE08E893FF22AB
:10300A0009E993C39D6008402974FB29F980F109F5
:10301A00E993C39E6008401A74FA29F980E209E923
:10302A0093D39F6008400B74F929F980D3191919B1
:10303A001919E9C313C313FF22740093F8ECC39858
:10304A004024701F740193F8EDC3984019701474EA
:0E305A000293F8EEC398400E7009740393F8C9
:10306800EFC39840037F00227F0122EDF8E6F008C5
:10307800A3DFFA22EDF8E0F608A3DFFA22E0A36363
:10308800A201F0A363A201DFF475A2002263A201EA
:10309800F0A363A20122E0A363A201F0A363A2014B
:1030A800E0A363A201F0A363A201E463A201F0A379
:1030B80063A201DFE175A20022E0A363A2016DFE15
:1030C800936CFDEE058393FC158363A201DFEA751B
:1030D800A200227F00E493A363A201F00F600CA377
:1030E800E583C2E3F58363A20180EA75A20022E0CA
:1030F800A363A201F0A3E583C2E3F58363A201DF22
:10310800EE75A20022E0A363A201F0A3E583C2E466
:10311800D2E3F58363A201DFEC75A20022E0A3638A
:10312800A201F0A3E58344F8C2E5F58363A201DFB9
:10313800EC75A20022E583C2E3F583E0A363A20154
:10314800F0A363A201DFEE75A20022E583C2E4D2F8
:0A315800E3F583E0A363A201F0A3F6
:1031620063A201DFEC75A20022E58344F8F583E057
:10317200A363A201F0A363A201DFEE75A20022F90C
:1031820022C002C004C00612FFF0D006D004D00252
:01319200221A
:1046A5004572724C656E210A000A496E49503A00FE
:1046B500205544502054696D654750530A00200A1F
:1046C500444154414752414D3A20002043414E2038
:1046D50054696D654750530A0020547261737353D2
:1046E500656E644552520A000ACEF8C4EBE8EDFB4C
:1046F50043414E210A000A45727241647243414E9C
:104705003A00205265496E69742043414E0A0020E3
:1047150043414E283029203E20544F210A00205481
:0C4725005520300A0020545520310A00B5
:03001E00E4FF22DA
:104F7900C2A9438902758C48758A4875D90475DBBD
:104F89004875DC4875DD4875DE48E4F5E9F5F9D280
:084F9900D9C2DAD28CD2DE226B
:104EA200C2D9906EDBE07013E5E92419F5EB30D737
:104EB20006E5F904F5FB2285F9FB22E5E924C8F5AC
:0E4EC200EB30D706E5F904F5FB2285F9FB225B
:104D0100C2D9906EDBE0702C302D16E5E92432F526
:104D1100EB30D707E5F904F5FB800385F9FBC22DDC
:104D210022E5E92405F5EB30D706E5F904F5FB2288
:104D310085F9FB22E5E92432F5EB30D706E5F904E4
:074D4100F5FB2285F9FB22BE
:104FA100124F79906EDBE0C3946450061240C31235
:104FB1004EA2125170D22CE4F556906FF3F0F545E4
:074FC100F55AC22DF558223C
:104D8A00EF24FCF545D3940D4010200B077E467F97
:104D9A00A5123C61E4F545D22A22906BB363A201C5
:104DAA00906FE363A201AF45123085C22A200B0D32
:0E4DBA007E467FAE7C6B7DB3AB45123A56222F
:0F510A00D3EF6480948D5006E55A70028F5A22BD
:10285B0020D903022930202C03022930E55A604A83
:10286B0090683E540FFF7D4712307CE54764017042
:10287B001E906846E0B4FF0ED22E200B127E467FD0
:10288B00B5123C618009302E06E4F55A022930124C
:10289B004EA2123E2A200B0D7E467FC37C687D3EE6
:1028AB00AB5A123A56E4F55A807BE5456043906F7C
:1028BB00E7E02405F527D3940D4007E4F545D22A2C
:1028CB008063906FE3E527540FFF7D4712307CE563
:1028DB004730E702D22DE547B40109302E06E54A11
:1028EB0064016003123E2A124EA2E4F545D22A80FF
:1028FB0034E557601E906EC7540FFF7D4712307C36
:10290B00E547B40103202E03123E2A124EA2E4F532
:10291B0057801220110C906EDBE0C39464500312AD
:10292B004949124EA21244618F27EF70030229E32B
:10293B00124D01E4F558E547547EB54703124C069A
:10294B00E547B4010CD22E200B077E467FD0123CFC
:10295B0061E559C394C8501B30031874DC2559F535
:10296B0082E4346EF583E5272559F5597D47AF276A
:10297B00123073300121E54720E71C906DB37D4782
:10298B00AF27123073AF27124315EF700A200B07D6
:10299B007E467FDE123C61E5475481703BE527D3D1
:1029AB00940D400C200B317E467FED123C6180284C
:1029BB00E549D39407401C200B1E90693F7D47AF20
:1029CB00271230737E467FFB7C697D3FAB27123A23
:1029DB00568005AF27122AFE300E1A300015906E66
:1029EB00DBE0C39464500C0558E55894F04004C2E6
:1029FB00AF80FEC20E200203022AF8E5566031D3E7
:102A0B009401400415568028906FF3E004F0E0D356
:102A1B009403400D200B077E477F07123C61124F3A
:102A2B00A1200B077E477F14123C61E4F556D22C94
:102A3B00302B43E557703F906EC704F0A37408F03A
:102A4B00A37480F0A37401F0A37406F0906FDEE022
:102A5B00906ECCF0906FDFE0906ECDF0906FE0E079
:102A6B00906ECEF0906FE1E0906ECFF0E4A3F0A308
:102A7B00F075570BC22B302972906FDCE07035E587
:102A8B00577031906EC77442F0A37408F0906FDDED
:102A9B00E0906EC9F0906FE2E0906ECAF0A3740103
:102AAB00F0755706200B077E477F23123C61906F12
:102ABB00DCE004F0906FDCE06402702FE557702BC4
:102ACB00906EC77402F0A37408F0906FDDE0906E07
:102ADB00C9F0A3F0A37401F0755706200B077E47CE
:102AEB007F2A123C61906FDCE004F0C202120026D8
:022AFB00C20017
:012AFD0022B6
:104E6F00E559602CE4906CAFF0A3E559F0906EB467
:104E7F00E0906CB1F0A37419F0906EDC63A2019016
:104E8F006CB363A201AF59123085E4F5597F01224B
:034E9F007F00226F
:0B514000302A05C22A7F01227F0022D6
:0100210022BC
:06516A00E4F559F54522B1
:0A514B00E490693FF0A3F0A3F02206
:0751630020457272210A00D1
:1050AC00EF600A7B10E4FD7F0C124F26227B107DF3
:0750BC00107F0C124F2622A9
:1040C300D29475C353C29475C5C0E5C4B480FB854F
:1040D300C528D2947DE07F0F125034906EDBE0440C
:1040E30080FD7F2A1250347D247F291250347D04B1
:1040F3007F28125034E4FD7F2B125034752A20E4BC
:10410300F529E4FDAF2A125034052A0529E529C310
:10411300940840EEE4F52AF529E4FDAF2A12503461
:10412300052A0529E529C3940C40EE7D087F051275
:104133005034752A10E4F529E4FDAF2A12503405F2
:104143002A0529E529C3940C40EE7D3C7F0C1250CF
:10415300347D077F0F1250347DFF7F2B125034754F
:104163002A30E4F528E4F529E4FDAF2A125034059A
:104173002A0529E529C3940E40EE052A052A0528B8
:10418300E528C3940340DE7D047F60125034E4FDD0
:054193007F70125034A2
:014198002204
:10501000C29475C503E5C4B480FBAEC58FC5E5C4B5
:10502000B480FBAEC5E4F5C5E5C4B480FBAEC5D223
:0350300094AF0634
:01503300225A
:10503400C29475C502E5C4B480FBAEC58FC5E5C492
:10504400B480FBAEC58DC5E5C4B480FBAEC5D294B7
:015054002239
:104F2600C29475C505E5C4B480FBAEC58FC5E5C49E
:104F3600B480FBAEC58BC5E5C4B480FBAEC58DC5DC
:094F4600E5C4B480FBAEC5D294B1
:014F4F00223F
:103F0A00C29475C503E5C4B480FBAEC5EF60047EF8
:103F1A007080027E608EC5E5C4B480FBAEC5E4F550
:103F2A00C5E5C4B480FB85C546E4F5C5E5C4B480DF
:103F3A00FB85C547E4F5C5E5C4B480FB85C548E4FF
:103F4A00F5C5E5C4B480FB85C549E4F5C5E5C4B447
:103F5A0080FB85C54AE4F5C5E5C4B480FB85C54B3D
:103F6A00E54B540FFE60741EE4F5C5E5C4B480FB4E
:103F7A0085C54CEE60651EE4F5C5E5C4B480FB85D5
:103F8A00C54DEE60561EE4F5C5E5C4B480FB85C593
:103F9A004EEE60471EE4F5C5E5C4B480FB85C54F07
:103FAA00EE60381EE4F5C5E5C4B480FB85C550EE65
:103FBA0060291EE4F5C5E5C4B480FB85C551EE60F1
:103FCA001A1EE4F5C5E5C4B480FB85C552EE600B44
:0D3FDA00E4F5C5E5C4B480FB85C553D29461
:013FE70022B7
:103E2A00906EDBE0C394644003023F07C29475C5F9
:103E3A0002E5C4B480FBAFC575C531E5C4B480FBE7
:103E4A00AFC5E54B540FFE8547C5E5C4B480FBAF4B
:103E5A00C58548C5E5C4B480FBAFC58549C5E5C479
:103E6A00B480FBAFC5854AC5E5C4B480FBAFC58540
:103E7A004BC5E5C4B480FBAFC5EE606C1E854CC56E
:103E8A00E5C4B480FBAFC5EE605E1E854DC5E5C4D2
:103E9A00B480FBAFC5EE60501E854EC5E5C4B48044
:103EAA00FBAFC5EE60421E854FC5E5C4B480FBAFCB
:103EBA00C5EE60341E8550C5E5C4B480FBAFC5EEBF
:103ECA0060261E8551C5E5C4B480FBAFC5EE6018F7
:103EDA001E8552C5E5C4B480FBAFC5EE600A8553A2
:103EEA00C5E5C4B480FBAFC5D2947F02C29475C540
:0F3EFA0081E5C4B480FBAFC5D29475560AC22CC3
:013F09002295
:104C0600C29475C502E5C4B480FBAFC575C541E560
:104C1600C4B480FBAFC58547C5E5C4B480FBAFC54A
:104C26008548C5E5C4B480FBAFC58549C5E5C4B4B0
:104C360080FBAFC5854AC5E5C4B480FBAFC5E4F5C6
:104C4600C5E5C4B480FBAFC5D2947F02C29475C5D6
:0A4C560082E5C4B480FBAFC5D29420
:014C60002231
:10494900C29475C502E5C4B480FBAFC575C551E510
:10495900C4B480FBAFC574872513F582E43461F5CF
:1049690083E0F5C5E5C4B480FBAFC575C508E5C4EA
:10497900B480FBAFC574882513F582E43461F583EF
:10498900E0F5C5E5C4B480FBAFC575C50FE5C4B492
:1049990080FBAFC50513051374872513F582E4342D
:1049A90061F583E07002F513E4F5C5E5C4B480FB55
:1049B900AFC5D2947F02C29475C584E5C4B480FBA7
:0449C900AFC5D29410
:0149CD0022C7
:104461003092037F00227F2C1250108F28E52830D4
:10447100E209D22CE4F556906FF3F0E52830E558C7
:10448100200B077E517F63123C617F2D1250108FEC
:1044910029200B11E528FE7C00E42529FFEC3EFED6
:1044A1007D03123D49E4FBAD297F2D124F26200BE0
:1044B1001BE52830E016E4FF123F0AE547FE7C00C9
:1044C100E4254BFFEC3EFE7D03123D49AB28E4FDA4
:1044D1007F2C124F267F0022E4F529E52830E00DDC
:1044E100E4FF123F0AE54B54072405F529AB28E404
:0844F100FD7F2C124F26AF29BC
:0144F90022A0
:10113D005452414E5A004D415842005254530044AE
:10114D00454C4159004D4F4445004B5000545500FE
:10115D0043414E004B565400415400444952004304
:10116D00414E4D4F4E00475254494D450054495440
:10117D0053005453494E5600003E2A2C312CCFE0DB
:10118D00F0E0ECE5F2F0FB20F3EFF0E0E2EBFFFE38
:10119D00F9E5E3EE20EAEEEDF2F0EEEBEBE5F0E053
:1011AD0020CACF20C8F1E5F2FC0A003E4C2C6B3072
:1011BD00312C25732C43EAEEF0EEF1F2FC20EDE03C
:1011CD0020F8E8EDE52043414E2C30202D20353020
:1011DD0030EAE1283530EC292C31202D203530EA4C
:1011ED00E128353030EC290A0030202D2035303003
:1011FD00EAE1283530EC290031202D203530EAE1A7
:10120D0028353030EC29003E532C6B30322C2562C2
:10121D00752CCCE0EAF12E20E0E4F0E5F120E1EBD5
:10122D00EEEAE020D2D128302D38290A003E532C89
:10123D006B30332C2562752CCCE0EAF12E20E0E4E6
:10124D00F0E5F120E1EBEEEAE020D2C8D228302D16
:10125D0038290A003E532C6B30342C2562752CCC6A
:10126D00E0EAF12E20E0E4F0E5F120E1EBEEEAE03A
:10127D0020D2D328302D38290A003E422C6330313C
:10128D002C2562752CC2F2EEF0E8F7EDFBE920EAB1
:10129D00EEEDF2F0EEEBEBE5F020EDE020F8E8ED11
:1012AD00E50A003E2A2C312CCFE0F0E0ECE5F2F01F
:1012BD00FB20EFF0EEF2EEEAEEEBE020C3F0E0ED16
:1012CD00E8F220EFEE20EFEEF0F2F320525332333E
:1012DD00320A003E432C61636B2C25732CCFEEF04C
:1012ED00FFE4EEEA20C0D4C10A00312DD2D128305E
:1012FD002B312920322DD2C8D228302920332DD29E
:10130D00D320342DD2C8D228312920352DD2D12841
:10131D00322B332920382DD2C8C8003E4C2C6B30CF
:10132D00352C256C752CD1EAEEF0EEF1F2FC20EEA9
:10133D00E1ECE5EDE020EDE020EFEEF0F2F32C3105
:10134D0030302C3230302C3330302C3630302C3194
:10135D003230302C323430302C343830302C393669
:10136D0030302C31393230302C33383430302C355C
:10137D00373630302C3131353230300A003E532C77
:10138D006B30362C2562752CCDEEECE5F020CACFF6
:10139D00200A003E422C6730312C2562752CCCE0A2
:1013AD00E3E8F1F2F0E0EBFC0A003E422C6730324C
:1013BD002C2562752CC8EDE2E5F0F2E8F0EEE2E0E6
:1013CD00F2FC20E7EDE0F7E5EDE8FF20D2D10A00D1
:1013DD003E422C6730332C2562752CC7E0EFF0E0D0
:1013ED00F8E8E2E0F2FC20E2F0E5ECFF20F1E5F0B8
:1013FD00E2E5F0E00A003E422C6730342C256275A0
:10140D002CC2FBF1F2E0E2EBFFF2FC205254532030
:10141D00EFF0E820EFE5F0E5E4E0F7E50A003E53F4
:10142D002C6730352C2562752CC7E0E4E5F0E6EA33
:10143D00E020EFE5F0E5E4E0F7E820EFEEF1EBE595
:10144D002052545320282A3130ECF1290A003C2136
:10145D00003C6B30313D003C6B30323D003C6B301D
:10146D00333D003C6B30343D003C6330313D003C3E
:10147D006B30353D003C6B30363D003C6730313DC7
:10148D00003C6730323D003C6730333D003C6730F7
:10149D00343D003C6730353D000ACFE5F0E5E4E032
:1014AD00F7E03A2000544949204379636C650A00FE
:1014BD005453204379636C650A0054530A00544910
:1014CD00540A005455204F4B0A005455204469616D
:1014DD00670A005455205265710A00205455205456
:1014ED00696D654F5554210A000ACFF0E8E5EC3AD5
:1014FD0020000A4352432045525221000AD7F3E6F9
:10150D00EEE920EDEEECE5F020CACF21000A5265A0
:10151D007154533120000A52657154533520000A1D
:10152D0052657154495420000ACFF0E8EDFFF2E006
:10153D0020EAEEECE0EDE4E020D2D320002020D232
:10154D00D320E7E0EDFFF2EE210A000ACDE520EF12
:10155D00EEEDFFEB20F2E8EF20EFE0EAE5F2E0211F
:10156D000A0000112332465765748C9DAFBECADB4D
:10157D00E9F810013322564775649C8DBFAEDACB66
:10158D00F9E82130021367764455ADBC8E9FEBFA16
:10159D00C8D93120120377665445BDAC9E8FFBEA46
:1015AD00D8C94253617004152736CEDFEDFC8899FA
:1015BD00ABBA5243716014053726DECFFDEC988926
:1015CD00BBAA6372405125340617EFFECCDDA9B8D6
:1015DD008A9B7362504135241607FFEEDCCDB9A806
:1015ED009A8B8495A7B6C2D3E1F008192B3A4E5FBA
:1015FD006D7C9485B7A6D2C3F1E018093B2A5E4FE6
:10160D007D6CA5B48697E3F2C0D129380A1B6F7E95
:10161D004C5DB5A49687F3E2D0C139281A0B7F6EC5
:10162D005C4DC6D7E5F48091A3B24A5B69780C1D79
:10163D002F3ED6C7F5E49081B3A25A4B79681C0DA5
:10164D003F2EE7F6C4D5A1B082936B7A48592D3C55
:10165D000E1FF7E6D4C5B1A092837B6A58493D2C85
:10166D001E0F0089129B24AD36BF48C15AD36CE5BD
:10167D007EF78108931AA52CB73EC940DB52ED6465
:10168D00FF76028B109926AF34BD4AC358D16EE751
:10169D007CF5830A9118A72EB53CCB42D950EF6645
:1016AD00FD74048D169F20A932BB4CC55ED768E131
:1016BD007AF3850C971EA128B33ACD44DF56E96025
:1016CD00FB72068F149D22AB30B94EC75CD56AE311
:1016DD0078F1870E951CA32AB138CF46DD54EB6205
:1016ED00F97008811A932CA53EB740C952DB64ED01
:1016FD0076FF89009B12AD24BF36C148D35AE56CE5
:10170D00F77E0A8318912EA73CB542CB50D966EFD0
:10171D0074FD8B029910AF26BD34C34AD158E76EC4
:10172D00F57C0C851E9728A13AB344CD56DF60E9B0
:10173D0072FB8D049F16A920BB32C54CD75EE168A4
:10174D00F37A0E871C952AA338B146CF54DD62EB90
:10175D0070F98F069D14AB22B930C74ED55CE36A84
:10176D00F1780008040C020A060E0109050D030BA1
:10177D00070FFF113DFF1143FF1148FF114CFF11E2
:10178D0052FF1157FF115AFF115DFF1161FF1165D6
:10179D00FF1168FF116CFF1173FF117AFF117FFFAD
:0217AD001185A4
:1050C300EF540F90176F93FEC454F0FEEFC4540FC8
:0450D300932EFF22F7
:0300230002458A09
:0B458A00C0E0C083C082C0D075D01814
:1045950030984EC298755E01AF99201644201209D5
:1045A500EF6402703CD2128038301A04C21A80229D
:1045B500BF0904D21A802ABF0205530B808022BF8F
:1045C5000310906614E50BF0630B80530B80C21249
:1045D500800F7437250BF582E43466F583EFF0051B
:1045E5000B309927301322906185E0FFE50CC39FBE
:1045F5004006C213D21D8011AF0C050C74372FF580
:0B46050082E43467F583E0F599C29968
:09461000D0D0D082D083D0E0327A
:10393D007BFF7A11798612229B906EDBE0701475F5
:10394D002FFF7530117531F67BFF7A1179B8122280
:10395D009B8012752FFF7530127531057BFF7A1123
:10396D0079B812229B7BFF7A127914906186E0F56B
:10397D002F12229B7BFF7A12793A906101E0F52F8D
:10398D0012229B7BFF7A127961906100E0F52F1274
:10399D00229B7BFF7A127987A211E433F52F122235
:1039AD009B7BFF7A1279B012229B752FFF75301217
:1039BD007531F77BFF7A1279E012229B906838E01F
:1039CD00FEA3E0FFC3E49FFFE49EFEAB07FA339531
:1039DD00E0F9F87F007E8C7D0A7C0012266C8F3218
:1039ED008E318D308C2F7BFF7A13792812229B7BA1
:1039FD00FF7A13798A906403E0F52F12229B7BFFE7
:103A0D007A1379A0A21EE4336401F52F12229B7B59
:103A1D00FF7A1379B7A219E433F52F12229B7BFF9E
:103A2D007A1379DDA214E433F52F12229B7BFF7AF2
:103A3D00147903A21BE433F52F12229B7BFF7A141A
:093A4D00792B85092F12229B221E
:103668007E147F5B12483FEF4E70037F0122E49087
:103678006EDBF07E147F5E12483FEF4E60151250ED
:1036880092BF3106906EDB740AF0BF3206906EDB93
:103698007464F07E147F6412483FEF4E600A124B48
:1036A800A9906186EFF080069061867402F07E141E
:1036B8007F6A12483FEF4E600A124BA9906101EFF2
:1036C800F080069061017402F07E147F7012483F0A
:1036D800EF4E600A124BA9906100EFF080069061EE
:1036E800007402F07E147F7612483FEF4E600D1290
:1036F8004BA9EC4D4E4F24FF92118002C2117E144B
:103708007F7C12483FEF4E6023124BA9A804A905FD
:10371800AA06AB077F007E8C7D0A7C0012266C12FD
:1037280026FE906838EEF0A3EFF0800A90683874AF
:10373800FFF0A374DCF07E147F8212483FEF4E60E6
:103748000A124BA9906403EFF08006906403740199
:10375800F07E147F8812483FEF4E600E125092EFB1
:1037680024D0640124FF921E8002C21E7E147F8E24
:1037780012483FEF4E600C125092EF24D024FF9273
:10378800198002C2197E147F9412483FEF4E600CD4
:10379800125092EF24D024FF92148002C2147E1497
:1037A8007F9A12483FEF4E600C125092EF24D024BB
:1037B800FF921B8002C21B7E147FA012483FEF4E6F
:0E37C8006007124BA98F098003E4F5097F000A
:0137D60022D0
:102DA100E4F527E52775F003A4247FF582E43417C1
:102DB100F583E493FB740193FA740293F912259558
:102DC1007003022FA9E4F529F52AF528746725284F
:102DD100F582E43469F583E0FF7003022FA4E5274F
:102DE10075F003A4247FF582E43417F583E493FBA3
:102DF100740193FA740293F985298275830012256F
:102E0100AEFEEFB50608752A010529022F9FE52AB6
:102E11007003022F9FEE6003022F9AE527B40F0083
:102E21004003022FA4902E2DF8282873022E5A0257
:102E31002EA1022EDA022EDF022FA4022F37022F3B
:102E4100A4022F0A022FA4022FA4022F64022F8EA4
:102E5100022F92022FA4022F9674672528F9E434D9
:102E610069FA7B01C0031B8B32753300753400E4B2
:102E7100F535D00312333D8F2E8E2D8D2C8C2BAB3F
:102E81002EAA2DA92CA82B7F007E8C7D0A7C0012F6
:102E9100266C1226FE906838EEF0A3EFF0022FA404
:102EA10074672528F582E43469F583E024D09061C4
:102EB10086F074682528F582E43469F583E024D02E
:102EC100906101F074692528F582E43469F583E0A5
:102ED10024D0906100F0022FA4D21B022FA47467AA
:102EE1002528F9E43469FA7B01C0031B8B32753361
:102EF10000753400E4F535D00312333D8F2E8E2D4D
:102F01008D2C8C2B8F09022FA474672528F9E434AA
:102F110069FA7B01C0031B8B32753300753400E401
:102F2100F535D00312333D8F2E8E2D8D2C8C2B90A9
:102F31006EDBEFF0806D74672528F9E43469FA7B64
:102F410001C0031B8B32753300753400E4F535D0B5
:102F51000312333D8F2E8E2D8D2C8C2B906403EF1D
:102F6100F0804074672528F9E43469FA7B01C003D5
:102F71001B8B32753300753400E4F535D003123301
:102F81003D8F2E8E2D8D2C8C2BD21E8016D2118032
:102F910012D214800EC219800AE4F52AF5290528F7
:082FA100022DCD0527022DA42D
:012FA9002205
:10319300C229C21CC218C217C215E4906837F0C214
:1031A3001F9066167405F0C22BE4F508FF7F40906C
:1031B30061B9E4F0A3DFFCE4FF7F20906617E4F03D
:1031C300A3DFFCE4FF74042FF582E43466F583E4A3
:1031D300F0740C2FF582E43466F583E4F00FBF0836
:1031E300E4E4F50DF50EF512F511906302F090632A
:1031F30001F0C213C21DC216C212C21AF50C9061AD
:1032030085F0F509F50BF55EC210C21B90683874A2
:10321300FFF0A374F4F0E4906403F0C21EC211C281
:1032230014D219906EDBF0123668EF6003122DA1F1
:10323300E4F5137E617F87906186E0F513E513C3A0
:1032430094014007E513D394084003E4F513E51311
:1032530060220FEFAC0670010E14F5828C8374C4E8
:10326300F015130FEFAC0670010E14F5828C83E595
:1032730013F080DA906101E0F513E513C394014084
:1032830007E513D394084003E4F513E51360220F15
:10329300EFAC0670010E14F5828C8374C8F015131D
:1032A3000FEFAC0670010E14F5828C83E513F080EA
:1032B300DA906100E0F513E513C394014007E513C9
:1032C300D394084003E4F513E51360220FEFAC0633
:1032D30070010E14F5828C8374C2F015130FEFACDA
:1032E3000670010E14F5828C83E513F080DA0FEF7C
:1032F300AC0670010E14F5828C83E4F08F828E830A
:10330300F0F513F59BC2ADF5C9D2CDD2CCC2C9C27B
:10331300CAF5CDF5CC906838E0F5CBA3E0F5CA85C6
:10332300CBCD85CACCD29ED29CD2CAC2ACC298C2E3
:093333009975B81075B710D2AC01
:01333C00226E
:1050D700E5106FFF90166F93650FF510EF90156F42
:0350E70093F50F2F
:0150EA0022A3
:024263008F2D9D
:10426500E4FC752E61752F02F510F50FFDEDC39574
:104275002D5017052FE52FAE2E7002052E14F58251
:104285008E83E0FF1250D70D80E3052FE52FAE2E6C
:104295007002052E14F5828E83E510F0852F828538
:1042A5002E83E50FF0052D052D7E677F37752E6171
:1042B500752F028F828E837402F00FBF00010E0CE2
:1042C500E4FDEDC3952D5038852F82852E83E0F9C9
:1042D50064026008E964036003B9090D8F828E8367
:1042E5007409F00FBF00010E0C8F828E83E9F00F69
:1042F500BF00010E0C052FE52F7002052E0D80C2A3
:0F4305008F828E837403F00FBF00010E0CAF0484
:014314002286
:03517000C2162242
:104DC8008F2C201335AF2C124263906185EFF020B1
:104DD8000B127E147FA6123C617E617F02E4FBAD5C
:104DE8002C123FE8301B057F011250ACE509600327
:0B4DF800F55B22E4F50CD213D29922E7
:022AFE008F281F
:102B0000E54724BE7003022D4924FA7003022CC14C
:102B100024046003022DA0E54830E703022BC530F2
:102B20000C077E147FB2123C61E54A6068E549C338
:102B300094024003022DA0E5497007E54A14F529E7
:102B40008006E54A241FF529E52975F004A424032D
:102B5000F582746335F0F5837D4C7F04123073E5A4
:102B60002975F004A42401F582746235F0F5837DA3
:102B7000507F0412307374F92549F582E43461F50D
:102B8000837481F074B92529F582E43461F5837486
:102B900001F0D21722300C077E147FBD123C617405
:102BA000042549F582E43466F5837401F0E549753E
:102BB000F004A42417F582746635F0F5837D4C7F0C
:102BC0000412307322E54B64086003022DA0E5492E
:102BD000C394044003022DA0300C077E147FC7125B
:102BE0003C61752801E54A5407FFE528A8070880DD
:102BF00002C333D8FCF5287408250EF50EB50D0672
:102C00007408250DF50DE54A547FFFE549C433549A
:102C1000E02FFE7400250EF582E43460F583EEF0BB
:102C2000E54AC394805022EF131313541FFFE54964
:102C300025E025E02F2417F582E43466F583E0FFD4
:102C4000E528F4FEEF5EF0802EE54A547FFF131373
:102C500013541FFFE54925E025E02F2417F582E4F2
:102C60003466F583E04528F07400250EF582E434DF
:102C700060F583E04480F07401250EF582E4346051
:102C8000F5837D4C7F04123073E551FEE550FF7CE7
:102C9000007D0A1225DBEF7405250EF582E4346011
:102CA000F583EFF07406250EF582E43460F583E5D4
:102CB00052F07407250EF582E43460F583E553F095
:102CC00022300C077E147FCB123C61E54A54E0644D
:102CD000407003022DA0E54A547FF529E549701D97
:102CE000E5291313543FFF7401A807088002C3337A
:102CF000D8FC4211906301E04511F08024E549645D
:102D0000016003022DA0E5291313543FFF7401A8AD
:102D100007088002C333D8FC4212906302E04512D8
:102D2000F0E54975F020A47C002529FFEC35F0FE84
:102D3000EF25E0FFEE33FE74042FF58274643EF558
:102D4000837D4CAF4B12307322E54AB40113300C33
:102D5000077E147FD0123C61E54D04906FF4F0C201
:102D600029E54AB40216240CF582E43466F583E5BD
:102D70004DF0300C077E147FD7123C61E54AB40356
:102D80001F240CF582E43466F583E54DF0300C0722
:102D90007E147FE0123C61302906906FDC7402F0F3
:012DA0002210
:10002600906403E070030208E130002F050A906631
:1000360016E0600214F0906837E0600214F0C20027
:10004600302918906184E004F0E0D3940A400C3023
:100056000C077E147FE8123C61C229E55BB40109F6
:10006600E4F55BF50CD213D29930130DE50AD3945F
:10007600064009C213D21D8003E4F50A301D0AC2E8
:100086001D301B05E4FF1250AC30130302053DE59D
:100096005B600302053D201E0620150302053DC2D6
:1000A60015301F29C21FE4906102F0A37408F09076
:1000B6006403E0906104F0906615E0906105F0A39A
:1000C60074FEF0A3748FF07F06124DC822906FF471
:1000D600E0FF6025E4906102F0A37408F0906403E9
:1000E600E0906104F0A37483F0A3EFF0E4A3F09032
:1000F6006FF4F07F06124DC822E50E650D700302FF
:100106000200906837E060030202DAE50D2408F584
:1001160028E4906102F0A37408F0906403E0906113
:1001260004F0A374F0F0A37406F0A37491F07406BF
:100136002528F582E43460F583E0906108F07407C1
:100146002528F582E43460F583E0906109F07401B6
:100156002528F582E43460F583E090610AF07402A4
:100166002528F582E43460F583E090610BF0740392
:100176002528F582E43460F583E090610CF0740480
:100186002528F582E43460F583E090610DF0740073
:100196002528F582E43460F583E0FF547FFEC3949E
:1001A60040500BEFC454F00490610EF080167400BA
:1001B6002528F582E43460F583E0FFC454F0240575
:1001C60090610EF074002528F582E43460F583E032
:1001D600FFEEC4540F90610FF0EF5480FF740525B5
:1001E60028F582E43460F583E02F906110F0906882
:1001F600377414F07F0F124DC82230186AE49061EC
:1002060002F0A37408F0906403E0906104F0A37414
:1002160041F0A37420F0752A61752B07E4F5287464
:10022600172528F582E43466F583E0F529301906AA
:10023600FF1250C38F29852B82852A83E529F0F486
:10024600FFE5822408F582E43583F583EFF0052B7C
:10025600E52B7002052A0528E528C3940840C07FCF
:1002660015124DC8C21822301C6AE4906102F0A330
:100276007408F0906403E0906104F0A37445F0A361
:100286007420F0752A61752B0775280874172528C0
:10029600F582E43466F583E0F529301906FF12503D
:1002A600C38F29852B82852A83E529F0F4FFE58211
:1002B6002408F582E43583F583EFF0052BE52B70F2
:1002C60002052A0528E528C3941040C07F15124D63
:1002D600C8C21C222017030203DD9061FAE0FF90DA
:1002E60061F9E04F5401D3940050030203DDE4F5B5
:1002F6002874B92528F582E43461F583E070030299
:1003060003CF74B92528F582E43461F583E4F090CF
:100316006102F0A37408F0906403E0906104F0A316
:1003260074F0F0A37403F0A37491F0E528C4540F9D
:100336002408A3F0E528540FA3F0E52825E025E0DE
:10034600F5282401F582E43462F583E090610AF031
:1003560074022528F582E43462F583E090610BF09F
:1003660074032528F582E43462F583E090610CF08D
:1003760074042528F582E43462F583E090610DF07B
:10038600E4A3F074032528F582E43463F583E09052
:10039600610FF074042528F582E43463F583E09058
:1003A6006110F074052528F582E43463F583E09046
:1003B6006111F074062528F582E43463F583E09034
:1003C6006112F07F11124DC8220528E528C394401A
:1003D60050030202F7C217906616E0704130143ED1
:1003E6007478F0E4906102F0A37408F0906403E07E
:1003F600906104F0A374F0F0E4A3F0A37490F0A36A
:100406007408F0E4A3F0A3F0A3F0A3F0A3F0A3F024
:10041600A3F0A3F0A3F0A3F07F11124DC822E508C4
:10042600C39404506FE50825E0FF7403A80708800D
:1004360002C333D8FCF528551165287053E528F416
:100446005211E4906102F0A37408F0906403E09006
:100456006104F0A374F0F0A37402F0A37491F0E5C4
:10046600082420A3F0E50833333354F875F002A4CA
:100476002404F582E5F03464F58363A201906109F2
:1004860063A2017F101230857F17124DC80508221E
:100496000508808AE508C394085076E50824FC25FB
:1004A600E0FF7403A807088002C333D8FCF528557B
:1004B6001265287058E528F45212E4906102F0A300
:1004C6007408F0906403E0906104F0A374F0F0A364
:1004D6007402F0A37491F0E50854032440A3F0E5F8
:1004E6000833333354F875F002A42404F582E5F09A
:1004F6003464F58363A20190610963A2017F10123F
:1005060030857F17124DC805085308072205088055
:1005160083E4F508201E20E4906102F0A37408F03D
:10052600906403E0906104F0A37490F0E4A3F0A358
:10053600F07F06124DC822906614E0FF7003020891
:10054600E1F529E4F0200B1F7E147FF6123C61E5ED
:100556002954802437F582E43466AF82FEE52954B7
:100566007FFDE4FB123FE8E52970030208E1E52977
:100576005480FF2437F582E43466AD82F52A8D2B4C
:10058600E4F510F50F8F28E528C395295018052B9B
:10059600E52BAE2A7002052A14F5828E83E0FF123F
:1005A60050D7052880E1E50F4510600E300B030299
:1005B60008E17E147FFF123C6122E529548024372E
:1005C600F582E43466AF82F52A8F2B7402252BF56B
:1005D6002BE4352AF52A852B82F583E0FF90640308
:1005E600E0FEEF6E600E300B030208E17E157F0918
:1005F600123C6122052BE52B7002052AF582852A1D
:1006060083E0FFB43003D21522EF640170030208C1
:10061600E1EF64187037906605E0FF906604E04FDE
:10062600600CD218200B077E157F1A123C6190666B
:1006360007E0FF906606E04F70030208E1D21C3027
:100646000B030208E17E157F23123C6122852B8273
:10065600852A83E0B41915200B077E157F2C123CE2
:1006660061906301E0F511A3E0F51222852B8285E6
:100676002A83E0FF54F064F0600302076990661570
:10068600EFF0052BE52B7002052AF582852A83E01B
:10069600FF64807033052BE52B7002052AF58285F1
:1006A6002A83E0644060030208E1D21F052BE52B94
:1006B6007002052AF582852A83E064086003020831
:1006C600E1D214906616F022EFB40127052BE52B34
:1006D6007002052AF582852A83E0644F60030208CA
:1006E600E1906837E070030208E17408250DF50D06
:1006F600E4F022852B82852A83E060030208E10567
:100706002BE52B7002052AF582852A83E064426078
:10071600030208E1052BE52B7002052AF582852ADE
:1007260083E0906FDEF0052BE52B7002052AF5823B
:10073600852A83E0906FDFF0052BE52B7002052AF2
:10074600F582852A83E0906FE0F0052BE52B700299
:10075600052AF582852A83E0906FE1F0D22BC21438
:10076600D21F22852B82852A83E0FF64116008EF61
:10077600641260030208BFE529547F640E60030219
:1007860008BF200B077E157F35123C6130290E30DD
:100796000B030208E17E157F4A123C6122852B82FB
:1007A600852A83E0540314F529052BE52B700205F1
:1007B6002AF582852A83E0F52830E709E4906FDD83
:1007C600F0906FE2F0E52830E60BE4906FDDF090F4
:1007D6006FE27410F0E52830E50B906FDD7401F0E0
:1007E600E4906FE2F0E52830E40C906FDD7401F0E0
:1007F600906FE27410F0E52830E30B906FDD740221
:10080600F0E4906FE2F0E52830E20C906FDD7402C0
:10081600F0906FE27410F0E52830E10B906FDD7414
:1008260003F0E4906FE2F0E52830E00C906FDD74A1
:1008360003F0906FE27410F07402252BF52BE4356B
:100846002AF52A852B82F583E0F52830E700E5288E
:1008560030E607906FE2E02402F0E52830E50790E5
:100866006FE2E02404F0E52830E407906FE2E0242C
:1008760006F0E52830E307906FE2E02408F0E5286B
:1008860030E207906FE2E0240AF0E52830E10790B5
:100896006FE2E0240CF0E52830E007906FE2E024F8
:1008A6000EF0906FE2E02529F0D229E4906184F001
:1008B600906FDCF0906FF4F022200B1F7E157F58AE
:1008C600123C61E52954802437F582E43466AF8210
:0B08D600FEE529547FFDE4FB123FE823
:0108E10022F4
:104625000217AFE493A3F8E493A34003F68001F2E5
:1046350008DFF48029E493A3F85407240CC8C33396
:10464500C4540F4420C8834004F456800146F6DF65
:10465500E4800B0102040810204080905155E47E4F
:10466500019360BCA3FF543F30E509541FFEE4935A
:10467500A360010ECF54C025E060A840B8E493A321
:10468500FAE493A3F8E493A3C8C582C8CAC583CA4C
:10469500F0A3C8C582C8CAC583CADFE9DEE780BE04
:01515B000053
:10259500BB010689828A83E0225002E722BBFE0244
:0925A500E32289828A83E4932277
:1025AE00BB010CE58229F582E5833AF583E02250E2
:1025BE0006E92582F8E622BBFE06E92582F8E2222C
:0D25CE00E58229F582E5833AF583E4932246
:1025DB00BC000BBE0029EF8DF084FFADF022E4CCE4
:1025EB00F875F008EF2FFFEE33FEEC33FCEE9DECAD
:1025FB00984005FCEE9DFE0FD5F0E9E4CEFD22EDF3
:10260B00F8F5F0EE8420D21CFEADF075F008EF2F3C
:10261B00FFED33FD4007985006D5F0F222C398FD2D
:05262B000FD5F0EA22CA
:1026300075F008758200EF2FFFEE33FECD33CDCC61
:1026400033CCC58233C5829BED9AEC99E5829840E4
:102650000CF582EE9BFEED9AFDEC99FC0FD5F0D6C1
:10266000E4CEFBE4CDFAE4CCF9A88222B800C1B9EB
:102670000059BA002DEC8BF084CFCECDFCE5F0CB29
:10268000F97818EF2FFFEE33FEED33FDEC33FCEB62
:1026900033FB10D703994004EB99FB0FD8E5E4F91D
:1026A000FA227818EF2FFFEE33FEED33FDEC33FC0A
:1026B000C933C910D7059BE99A4007EC9BFCE99AFE
:1026C000F90FD8E0E4C9FAE4CCFB2275F010EF2F43
:1026D000FFEE33FEED33FDCC33CCC833C810D70743
:1026E0009BEC9AE899400AED9BFDEC9AFCE899F87E
:0E26F0000FD5F0DAE4CDFBE4CCFAE4C8F92211
:0E26FE00C3E49FFFE49EFEE49DFDE49CFC22ED
:10270C00EB9FF5F0EA9E42F0E99D42F0E89C45F023
:01271C00229A
:0C271D00ECF0A3EDF0A3EEF0A3EFF0222F
:10272900A8828583F0D083D08212274012274012D5
:102739002740122740E473E493A3C583C5F0C583FA
:10274900C8C582C8F0A3C583C5F0C583C8C582C8FA
:01275900225D
:10223900E53B242FF8E6053B22782C302702782F3E
:10224900E475F0011227BB0225952020EB7F2ED2E1
:10225900208018EF540F2490D43440D4FF30240B3D
:10226900EF24BFB41A0050032461FFE53C60021556
:102279003C053FE53F7002053E30270D782CE4759B
:10228900F0011227BBEF02275A024CBA7403D22776
:102299008003E4C227F53B8B2C8A2D892EE4F53C7B
:1022A900F53EF53FE53C60077F2012227480F57505
:1022B9003DFFC221C220C222C223C225C226C22892
:1022C900122242FF700D3027057F00122285AF3F91
:1022D900AE3E22B4255FC2D5C224122242FF24D0C9
:1022E900B40A00501A75F00A783C30D50508B6FFD3
:1022F9000106C6A426F620D5047002D22380D9246B
:10230900CFB41A00EF5004C2E5D224022485D221A9
:1023190080C6D22080C0D22280BCD2D580BAD22534
:1023290080B47F201222742022077401B53C00403A
:10233900F1122239FF1222740222ADD228D226804C
:1023490095122239FB122239FA122239F94A4B70B5
:102359000679567A257BFF20222EE53C602A7E00ED
:102369008E827583001225AE60060EEE653D70F013
:10237900C2D5EBC0E0EAC0E0E9C0E0EE1224CCD05F
:10238900E0F9D0E0FAD0E0FB122595FF60AAEBC096
:10239900E0EAC0E0E9C0E0122274D0E02401F9D0FB
:1023A900E03400FAD0E0FBE53D0460DCD53DD9809E
:1023B900877BFF7A2479C8D222809C7910800279A0
:1023C90008C226C2288008D2D5790A8004790AC2AF
:1023D900D5E53D047002F53DE4FAFDFEFF12223910
:1023E900FC7B08202113122239FD7B1030200A12B0
:1023F9002239FE122239FF7B20EC3382D592D55047
:1024090013C3E43020069FFFE49EFEE42021039DD0
:10241900FDE49CFCE4CBF8C221EC700CCFCECDCC12
:10242900E824F8F870F38017C3EF33FFEE33FEEDBD
:1024390033FDEC33FCEB33FB994002FB0FD8E9EB9E
:10244900302105F8D0E0C448B221C0E00AEC4D4E75
:102459004F78207B0070C2EAB53D0040BCC0E01255
:1024690024CED0F0D0E0202104C4C0E0C4B221C001
:10247900F012225DD0F0D5F0EB0222AD12281A231A
:102489004A5323C458231B4C23174223C84F23D034
:0F2499004423D04923304323D65523BA4623BAD0
:1024A8004523BA47257650231F2D23232E23462B59
:1024B800232723234420255F2A22DF480000233EC8
:1024C8003F3F3F00790AA2D5202314302509B910CF
:1024D800020404B9080104A2D520260250010420F0
:1024E80022689222B53C005034C0E07F2030231986
:1024F8007F30A22272267225500F122525C222C2D1
:1025080026C225C2287F30800F302503E9C0E0129B
:102518002274302503D0E0F9D0E0B53CCC30251743
:102528007F30B9100C1222747F583024077F7880CE
:1025380003B908031222743022057F2D0222747F0A
:10254800202028F87F2B2026F322922280CF286E85
:10255800756C6C2900D2211222393021F8C22178F9
:102568003C30D50108F60222DF2D5043495812228B
:10257800392403B405004001E490257193122265C3
:0D258800743A122265D223753C040223C46C
:10333D008B2F8A308931E4F53BF53AF539F538F5BF
:10334D0036F537E533453445326012EBC0E0EAC05F
:10335D00E0E9C0E0AB32AA33A9341227CBAB2F057D
:10336D0031E531AA307002053014F9122595F53C7E
:10337D00C394094007E53CD3940D40E1E53C64203E
:10338D0060DBE53CB42D054337038016E53CB42BDB
:10339D0005433701800C74FF2531F53174FF35304D
:1033AD00F530E53560046410703FAB2FAA30A931BC
:1033BD0012259564306009E535702E75350A802922
:1033CD009000011225AEFF64786004EFB4581343EA
:1033DD00370175351074022531F531E43530F5308E
:1033ED008007E5357003753508AB2F0531E531AA3A
:1033FD00307002053014F9122595F53CC3946140E7
:10340D000AE53CD3947A5003533CDF74D0253CF548
:10341D003CC3940A400CE53C9411406D74F9253C75
:10342D00F53CE53CD395355060433701853B4085F0
:10343D003A3F85393E85383DAF357E00E4FCFDAB26
:10344D003BAA3AA939A83812276CC8ECC8C9EDC9EE
:10345D00CAEECACBEFCBE4FCFDFEEB253CF53BEE13
:10346D003AF53AED39F539EC38F538AF3BAE3AADC2
:10347D0039FCAB40AA3FA93EA83DD312270C5003FF
:10348D000233F64337040233F6E53720E003E480D8
:10349D002DE53345344532601EAB2FE53124FFF960
:1034AD00E53034FFFAEBC0E0EAC0E0E9C0E0AB3252
:1034BD00AA33A9341227CBE53730E20774FFFFFE9C
:1034CD00FDFC22E537AF3BAE3AAD39AC3830E10308
:0434DD000226FE22A3
:10275A00BB010689828A83F0225002F722BBFE015E
:02276A00F32258
:10276C00E88FF0A4CC8BF0A42CFCE98EF0A42CFC0C
:10277C008AF0EDA42CFCEA8EF0A4CDA8F08BF0A48A
:10278C002DCC3825F0FDE98FF0A42CCD35F0FCEBE9
:10279C008EF0A4FEA9F0EB8FF0A4CFC5F02ECD39AE
:0F27AC00FEE43CFCEAA42DCE35F0FDE43CFC221B
:1027BB00FAE6FB0808E6F925F0F618E6CA3AF6221F
:1027CB00BB011A89828A83D0F0D0E0F8D0E0F9D02F
:1027DB00E0FAD0E0FBE8C0E0C0F00228495016E96F
:1027EB00F8D083D082D0E0F9D0E0FAD0E0FBC08201
:1027FB00C083022840BBFE16E9F8D083D082D0E01C
:0F280B00F9D0E0FAD0E0FBC082C083022852224D
:10281A00D083D082F8E4937012740193700DA3A34D
:10282A0093F8740193F5828883E473740293686061
:06283A00EFA3A3A380DF61
:09284000EBF608EAF608E9F622BD
:09284900EBF0A3EAF0A3E9F02290
:09285200EBF208EAF208E9F222B7
:00000001FF
